:020000020000FC
:020000000EC030
:0200120026C006
:10001C00189504E00EBF0FE50DBF00E007BB0EEF17
:10002C0008BB0EEF04BB00EE05BB0FEF01BB00E8F5
:10003C0002BB0EEF04BB00EE05BB05E003BF02BF25
:10004C0009B7016009BF05E106B975E090E880E0E9
:10005C007894FFCF0F930FB70F930CEF02BF7A95E5
:10006C0009F475E0713009F44AD0723009F44DD0BE
:10007C00733009F452D0743009F457D07530D9F577
:10008C005AD08395803509F036C0882700E0CAD055
:10009C00BD2FAC2F00E0C6D08894AC1FBD1F00E074
:1000AC00C1D08894AC1FBD1F00E0BCD08894AC1F9D
:1000BC00BD1F00E0B7D08894AC1FBD1F00E0B2D0CC
:1000CC008894AC1FBD1F00E0ADD08894AC1FBD1F41
:1000DC0000E0A8D08894AC1FBD1F8894B795A79555
:1000EC008894B795A7958894B795A795DB2FCA2FB9
:1000FC00D37026D036D00F910FBF0F9118951BD00F
:10010C00032F63D002BBA998089515D0042F5DD09E
:10011C0002BB90FD979AAA9808950DD0052F55D043
:10012C0002BB90FF979AAB98089505D0062F4DD03F
:10013C0002BBAC980895A99AAA9AAB9AAC9A089566
:10014C0090FD07C0D33061F4CC3F50F09160B89A69
:10015C0007C0D03029F4C43608F002C09E7FB8988E
:10016C00089590FD09C0D33039F4CF3F29F460E0F5
:10017C005BE04CE03DE028C0662755274427332739
:10018C006395C85ED340E0F708EEC00F03E0D01FC4
:10019C006A955395C456D040E0F704E6C00F00E0D2
:1001AC00D01F5A954395CA50D040E0F70AE0C00FD3
:1001BC0000E0D01F4A953395C150D04098F701E02C
:1001CC00C00F00E0D01F3A9508951FE3003041F1B5
:1001DC0016E0013029F11BE5023011F11FE4033068
:1001EC00F9F016E60430E1F01DE60530C9F01DE724
:1001FC000630B1F017E0073099F01FE7083081F0B6
:10020C001FE6093069F010E40A3051F011E70B30A9
:10021C0039F018E30C3021F01CE50D3009F010E03A
:10022C00012F08950F93379A0770006C07B97894D3
:10023C00339A00E905BF8895349AC4B1D5B10F91B2
:02024C00089513
:00000001FF
